:100000003F288F00220884002009282084138F08AD
:1000100003193A28F03091000E0880389000F03033
:1000200091030319910003198F0303193A28182823
:100030002B2003010C1820088E1F20088E0803199E
:100040000301900F252880060C28262800000F2881
:10005000841780053A280D080C0403198C0A803097
:100060000C1A8D060C198D068C188D060D0D8C0D35
:100070008D0D3A2883130313831264000800640073
:10008000061C4628061583160611831264000618FE
:100090004D2806118316061183126400861C5C2805
:1000A0000630A2000830A00064308E00233001200A
:0E00B00032308E00233001203F2863005D288F
:02400E00FD3F74
:00000001FF
